:0200000037289F
:10000800F80003088301EB000408EC000A08ED007F
:100018008A017908F1007A08F0007B08F3007C086F
:10002800F2007D08EF007E08EE007F08F4008301EF
:10003800871419278C1087107108F9007008FA00C6
:100048007308FB007208FC006F08FD006E08FE00D4
:100058007408FF006C0884006D088A006B08830030
:10006800F80E780E0900D22EF900FD010310FD30BC
:100078007A07031C5F28FC01F0307A05031D472826
:100088000430FC00FA0EFB010310FC0AFA0D031CF5
:100098004928FA0C7A0879020318F900FB0DFC0BC1
:1000A8004D28FD1F5928FB09FB0A7B08FD1F080086
:1000B800F909F90A0800FA0C03186828FA0C031C55
:1000C800F9010310F90C031C03107908FB00F9016E
:1000D800F90D5528FF01FD01FE017B087C04031D75
:1000E8007828F901FA0100341F30FF040310FF0AD1
:1000F800FB0DFC0D031C7B28FC0CFB0C7C087A0216
:10010800031D88287B087902031C90287B08F902C4
:100118007C08031C7C0AFA02FD0DFE0DFF0BFF1A7A
:100128008028FF1F9C28FD09FD0A0319FE03FE090C
:100138007D08FB007E08FC007F1F0034F909F90ADE
:100148000319FA03FA09003483010518C928D10AEA
:100158000319D20AC108031DBA285108053A5204E6
:10016800031DBA28C101C10AD101D201410BD82807
:100178005208023A943003195106031DD828023058
:10018800C100D101D201B927D828D101D201D12883
:10019800C101C424D828C101D8284108013A03194B
:1001A800CC28033A0319CF288518EB28D30A03195A
:1001B800D40AC208031DEE285308053A5404031D47
:1001C800EE28C201C20AD301D4012326EE28D301A6
:1001D800D401C20105191F29D50A0319D60AC30873
:1001E800031D00295508053A5604031D0029C301BB
:1001F800C30AD501D6017B25430B0D295608023ABF
:10020800943003195506031D0D290230C300D5018A
:10021800D6014308023A031915294308033A031D76
:10022800222955086E3A5604031D22290330C300BB
:10023800D501D6012229D501D601C3018519532933
:10024800D70A0319D80AC408031D34295708053AE0
:100258005804031D3429C401C40AD701D801222532
:10026800440B41295808023A943003195706031DD4
:1002780041290230C400D701D8014408023A0319C1
:1002880049294408033A031D562957086E3A580469
:10029800031D56290330C400D701D8015629D701B8
:1002A800D801C401051A6929D90A0319DA0AC50847
:1002B800031D6C295908053A5A04031D6C29C50108
:1002C800C50AD901DA01F9236C29D901DA01C50176
:1002D80008188C29DB0A0319DC0AC608031D7D29C6
:1002E8005B08053A5C04031D7D29C601C60ADB01CB
:1002F800DC01460B9B295C08023A943003195B0623
:10030800031D9B290230C600DB01DC01E3279B2982
:10031800DB01DC019429C601D7279B29C6019B294B
:100328004608013A03198F29033A031992298818B4
:10033800BA29DD0A0319DE0AC708031DAC295D08BE
:10034800053A5E04031DAC29C701C70ADD01DE01B9
:10035800470B08005E08023A943003195D06031D36
:1003680008000230C700DD01DE01DD2FDD01DE01FE
:10037800C129C701E92FC70108004708013A031935
:10038800BD29033A031D0800BF2932308301480202
:1003980003180800081A262A071A022A3808240609
:1003A800031DDE2939082506031DDE29BA08031DA9
:1003B800DE290716A01FEC2938083B06031DEC2987
:1003C80039083C06031DEC29BA08031DEC29071659
:1003D800071E282AA01339082907A8003808A700EB
:1003E8003C302802031C282AC430A807A70A183062
:1003F8002702031C282AE830A707282A38082706D6
:10040800031D0B2A39082806031D0B2A0712260884
:10041800023A03190712260B282A0712A0173908CF
:100428002A07BC003808BB003C303C02031C282AC1
:10043800C430BC07BB0A18303B02031C282AE8302A
:10044800BB07282A0712A013A601881A812A871A2F
:100458005D2A38082B06031D392A39082C06031D86
:10046800392ABA08031D392A8716211C472A380851
:100478003D06031D472A39083E06031D472ABA08C8
:10048800031D472A8716871E832A2110390830073B
:10049800AF003808AE003C302F02031C832AC4305A
:1004A800AF07AE0A18302E02031C832AE830AE07C5
:1004B800832A38082E06031D662A39082F06031DCD
:1004C800662A87122D08023A031987122D0B832AF0
:1004D8008712211439083107BE003808BD003C30A6
:1004E8003E02031C832AC430BE07BD0A18303D02F1
:1004F800031C832AE830BD07832A87122110AD0127
:10050800081B9A2A38084B06031D922A39084C06FC
:10051800031D922ABA08031D922A071738084906AC
:10052800031D9B2A39084A06031D9B2A0713881BAB
:10053800B22A38084F06031DA92A39085006031D98
:10054800A92ABA08031DA92A871738084D06031DCA
:10055800080039084E060319871308008713080096
:1005680083012012201B2016323048020318C02AAB
:100578002015A0154808C92A2011201FC42A2015B3
:10058800A011201BA0154808CE3EE600392B3908DB
:10059800E7003A08E800E9013808602E2508E70076
:1005A8003D30E800E9012408602E2908E7003E30C4
:1005B800E800E901E90A003060260F30B3000800BE
:1005C8002A08E7003F30E800E901E90A0030602620
:1005D8000F30B30008002C08E7004730E800E901B5
:1005E8002B08602E3008E7004830E800E901E90AE6
:1005F800003060260F30B30008003108E7004930AA
:10060800E800E901E90A003060260F30B30008006D
:100618004C08E7005130E800E9014B08602E4A0811
:10062800E7005230E800E9014908602E5008E70069
:100638005B30E800E9014F08602E4E08E7005C30A7
:10064800E800E9014D08602E4008E7006330E80043
:10065800E901E90A3F0860262011A118362BA010ED
:10066800A0120800A014A01608006608003A031992
:10067800CB2A0B3A0319D22A073A0319D92A013A85
:100688000319E42A183A0319EF2A033A0319F62A38
:10069800013A0319012B083A03190C2B3F3A0319A5
:1006A800132B093A03191A2B033A0319212B1B3A66
:1006B800031D0800282B00307427A400013074277C
:1006C800A50002307427AB0003307427AC00043057
:1006D8007427CB0005307427CC0006307427C90076
:1006E80007307427CA0008307427CF0009307427F0
:1006F800D0000A307427CD000B307427CE000C30A0
:100708007427A9000D307427AA000E307427B00092
:100718000F307427B10010307427BF0011307427D0
:10072800C00012307427E600660CA1100318A1144B
:1007380018302402031CA22B0730A4003C302502E9
:100748000318A50118302B02031CAC2B0930AB0091
:100758003C302C020318AC0118304B02031CB62B9A
:100768000C30CB003C304C020318CC011830490245
:10077800031CC02B0D30C9003C304A020318CA01C3
:1007880018304F02031CCA2B0E30CF003C305002E9
:100798000318D00118304D02031CD42B0F30CD00A4
:1007A8003C304E020318CE013C302902031CDE2BDC
:1007B8003B30A9003C302A02031CE42B0530AA0078
:1007C8003C303002031CEA2B3B30B0003C30310295
:1007D800031CF02B0A30B10018303F020318BF0188
:1007E800643040020318C00108002D2C2030C800D6
:1007F80008001F30C80008002A30C8000800293047
:10080800C8000800A115BA0108003E30C800080059
:100818003F30C80008003D30C80008004830C80014
:1008280008004930C80008004730C80008005230A6
:10083800C80008005130C80008005C30C800080033
:100848005B30C8000800A1182B2CA1140800A110C7
:1008580008008312031348081F3A0319FA2B3F3A7A
:100868000319FD2B093A0319002C033A0319032C29
:10087800183A0319062C0F3A0319092C033A0319DD
:100888000C2C013A03190F2C783A0319122C0F3A41
:100898000319152C013A0319182C183A03191B2CA3
:1008A800033A03191E2C093A0319212C073A031994
:1008B800242C3F3A031D0800272C83010910E60168
:1008C800E60A1E306602031C642C2014942C32089D
:1008D8008600B208031DA72C2010A72C0A3033026B
:1008E800031C7B2C20100030201910307F2C003086
:1008F800201910303307203E922C3408403E922CA9
:100908000030A01910303507603E922C3608803E22
:10091800922C0030201A10303707A03E8600A72CF2
:100928002208003A03196B2C013A0319722C033A76
:100938000319812C013A0319842C073A03198A2CCC
:10094800013A03198D2CE601E60A1E306602031CE3
:10095800A82C201CB12C0914B22C091083120313E3
:10096800A20A2208063A0319A201A01CBD2C891468
:10097800BE2C8910A01EC22C0915080009110800F8
:10098800E52C0B30C80008001530C80008001F30DF
:10099800C80008002930C8000800C80108003D3018
:1009A800C80008004730C80008005130C8000800D7
:1009B8005B30C80008003230C8000800D425C801E0
:1009C8000800831203134808003A0319C52C0B3A90
:1009D8000319C82C1E3A0319CB2C0A3A0319CE2C3A
:1009E8003F3A0319CE2C093A0319D12C033A0319BB
:1009F800D12C183A0319D32C0F3A0319D62C033AE1
:100A08000319D62C013A0319D62C783A0319D92C94
:100A18000F3A0319D92C013A0319D92C183A03199A
:100A2800DC2C033A0319DC2C093A0319DF2C073AAA
:100A38000319DF2C3F3A031D0800E22C532D390817
:100A48003427B900080025083427A500080029081C
:100A58003427A90008002A083427AA0008002C080F
:100A68003427AC00080030083427B00008003108EB
:100A78003427B10008004C083427CC0008004A0885
:100A88003427CA00080050083427D00008004E0850
:100A98003427CE00080040083427C000080083121D
:100AA80003134808323A0319232D0F3A0319272D47
:100AB800033A03192B2D013A03192F2D783A0319FC
:100AC800332D0F3A0319372D013A03193B2D183AE4
:100AD80003193F2D033A0319432D093A0319472DEA
:100AE800073A03194B2D3F3A031D08004F2DAC2D33
:100AF80039089527B900080025089527A50008009A
:100B080029089527A90008002A089527AA0008009F
:100B18002C089527AC00080030089527B00008007D
:100B280031089527B10008004C089527CC0008002B
:100B38004A089527CA00080050089527D0000800E1
:100B48004E089527CE0008004008A127C0000800DD
:100B5800831203134808323A03197C2D0F3A0319FC
:100B6800802D033A0319842D013A0319882D783A08
:100B780003198C2D0F3A0319902D013A0319942D5E
:100B8800183A0319982D033A03199C2D093A0319A9
:100B9800A02D073A0319A42D3F3A031D0800A82DDC
:100BA80083012408E6000030F9262508E600013014
:100BB800F9262B08E6000230F9262C08E600033057
:100BC800F9264B08E6000430F9264C08E600053003
:100BD800F9264908E6000630F9264A08E6000730F3
:100BE800F9264F08E6000830F9265008E6000930D3
:100BF800F9264D08E6000A30F9264E08E6000B30C3
:100C0800F9262908E6000C30F9262A08E6000D30F6
:100C1800F9263008E6000E30F9263108E6000F30D4
:100C2800F9263F08E6001030F9264008E6001130A2
:100C3800F9260030A1180130E6001230F92E442EB2
:100C48003808CE27B80008002408CE27A4000800DA
:100C58002B08CE27AB0008004B08CE27CB00080096
:100C68004908CE27C90008004F08CE27CF00080042
:100C78004D08CE27CD0008003F08CE27BF0008004A
:100C8800831203134808323A0319242E0F3A031922
:100C9800282E7A3A03192C2E163A0319302E033AC5
:100CA8000319342E093A0319382E073A03193C2E32
:100CB8003F3A031D0800402E8301EA00E9080319A2
:100CC8000819772E0C306A0203186D2EA014A01292
:100CD800712EA010A016F430EA07EA08031D792E39
:100CE8000C30EA00792EA010A0120A30FA006A0827
:100CF8003820B2000A30FA003208AD276A02B30081
:100D08000A30FA0067083820B4000A30FA003408BC
:100D1800AD276702B5000A30FA0068083820B60027
:100D28000A30FA003608AD276802B70008008301C8
:100D3800201BA12E87152017A52E871120136127A8
:100D4800C9216430FB00FC013F08F900FA014C2777
:100D580040087D07E3007E0803187E0AE400630468
:100D6800031908006408FC006308FB001030F90050
:100D78000E30FA006E207D08E1007E08E200DF0AEE
:100D88000319E00A6002031DCB2E61085F02031CF1
:100D9800080021150714DF01E0010800063083165A
:100DA80003139F00860187018901831209108701B7
:100DB800C101C201C301C401C501C601C7010F3089
:100DC80092007F308316920002308C00C0308B0076
:100DD800C42707156124A82086270711E501E50A1D
:100DE800783065020318ED2EF32E8301E700831691
:100DF80003178C18FB2E83120313670803178D0043
:100E08000313660803178C0083168C1303108B1BBF
:100E180003148B130C1555308D00AA308D008C14DB
:100E28000C1103188B17830108008301A30AA11D65
:100E3800212FA30187112013A1112308211D2F2F72
:100E48000A3A031D2E2F21110710A1182D2FA30ACE
:100E58002E2FA3032308643A031D0800A3019B2E29
:100E68008301E7000A30FA0067083820E60003101B
:100E7800660DE607E6070310E60D6608E702E70ACF
:100E88000A3067020318E7016608E70767080800E1
:100E9800FD01FE010310FC0CFB0C031C5A2F790802
:100EA800FD077A0803187A0AFE070310F90DFA0DF0
:100EB8007B087C04031900344E2F8301BA0A3A08D0
:100EC8003C3A031D0800BA01B90A39083C3A031D27
:100ED8000800B901B80A3808183A0319B801080017
:100EE8008301E700831603178C18762F83120313E8
:100EF800670803178D0083168C130C1483120C08D3
:100F0800031308008301C808031DB42A4308033AE1
:100F1800031DB42A4408033A031DB42A6330C800E9
:100F2800B42A8301E6000A30E6073C306602031C57
:100F38009F2FC430E607660808008301E6000A30E0
:100F4800E60764306602031CAB2F9C30E607660890
:100F58000800F90000307A1879070310F90D03101A
:100F6800FA0CFA0803190800AF2F3230830148023F
:100F78000318C12F3230C8070800D425C80108005B
:100F88005F23B801B901BA01A601AD01A013211070
:100F9800C80108008301E600E60A18306602031853
:100FA800E601660808008301071E0800A601A60AD4
:100FB80008008301871E08000230AD000800830185
:100FC800071E08000230A60008008301871E0800DB
:060FD800AD01AD0A0800A6
:02400E00313F40
:1042000007000000090000000C0000000D00000085
:104210000E0000000F0000003B0005003B000A00FC
:10422000000000000000FF00FF0001000300040088
:00000001FF
